:1018000000000000C034060041B00800CB0000001A
:02181000903115
:1080000055425C0135D0085A82452C243140006429
:108010003F4000000F93082492422C245C012F83E0
:108020009F4F488B0024F8233F402C000F930724D8
:1080300092422C245C011F83CF430024F923B240D9
:10804000805A5C01E2D26A02B240CD406C013F40EE
:108050004C011F83FE230343034382436E013F40D1
:1080600020001F83FE2303430343B2B26E01F523B6
:1080700082430201B24055006801F2D010002A028A
:10808000F2D010002402B2430402B2432602F240AE
:10809000BCFF4602F24040004402F24043004A0264
:1080A000F2434B02F2436602F24032006302F243B3
:1080B0006502F2438602B240200004093E400300FC
:1080C0003F40D1081F83FE231E83FC238243040903
:1080D000D243001CD243401CE2430A2492420018BF
:1080E0000C24924202180E24924204181024924248
:1080F0000618122492420818142492420A181624D0
:1081000092420C18182492420E181A249242101807
:108110001C24F240030022241F42B0013FB000049F
:10812000FB23B240A300B0011F42B0013FB00004E6
:10813000FB23D2423E8B1007D2423F8B1107D24223
:10814000408B1207D242418B1307D242428B140755
:10815000D242438B1507D242448B1607D242458B3D
:108160001707D242468B1807D242478B1907B240F5
:1081700000010C07B24022000407B2403E02020791
:10818000B240F3610007B240F00280071F4280074F
:108190003FB00002FB23B240F00290071F4290075D
:1081A0003FB00002FB23B012F68392421024002459
:1081B000924212240224B24080E92006824326061D
:1081C000F2D030006B02B0125282B2402896000901
:1081D00082430209B24080000409B2400018080935
:1081E000B2B20809FD27B24011021209B2400003E1
:1081F0001009824314093F406A0A1F83FE231F426D
:1082000014090F93F62392D30209B0124A83A2D322
:10821000020932D2FF3F32D0F000FD3F30403A8AAF
:10822000F2F0FDFF63020E4F8E104E4EC24E2E0630
:108230005E423D062EF3FC27C24F2E065F423D06EE
:108240002FF3FC275F422A061FF3FC23E2D36302CD
:1082500030411B153F402020B01220821B420024D9
:108260001A4202240F4B3FF0FF3F3FD00040B012B4
:1082700020820E4B0F4A8E108F104EEF0EEF8F1193
:108280000F110E100F110E100F110E100F110E10F6
:108290000F110E100F110E100F4E3FD00040B012F4
:1082A00020821A1730410B124F9327384E4F5E0A27
:1082B0003E5080235B422F091D434C4F7CF00F0042
:1082C00015204BCDC24B2F094F930E24CE430000F7
:1082D000CE430100CE430500FE4080FF0200FE4079
:1082E00080FF0600CE4307003B4130410D5D7C53CB
:1082F000E8270D5D7C53FA23E43F7FF07F004E4F6B
:108300005E0A3E50C0235B422E091D434C4F7CF059
:108310000F0004204BCDC24B2E09D63F0D5D7C5380
:10832000FD23F83F0B12C2430B241B434F4B7FD05E
:1083300080FFB012A6824F4BB012A6821B533B9215
:10834000F523C2431E243B413041C2433C09C24392
:108350003F0982430424C2430824C2432F09C24375
:108360002E09F24080FF2309F2408CFF2209F240DF
:1083700080FF2109F2408CFF2009B0122483D243F0
:108380002F09D2432E09F2F07F006302F240400031
:108390003C09C2433E09F240C4FF3D0930412B1560
:1083A0001A4204240B4A3A90090001383B42194210
:1083B00006240D4B0E493F407823B0125689095BC5
:1083C000824906240A8B824A0424C24B21092917B8
:1083D00030415C4286234C4C5D4287234D4D8D10CD
:1083E0000DDC0D9E012C0E4D824F0624824E04247E
:1083F000B0129E8330411B151B421C24824B02028B
:108400001A420C24824A84071F420E243FE31F5362
:10841000824F9407B2B0800046012C203D401200EC
:108420003E400C243F400018B01236890F9322249E
:10843000B24000A54401B24002A54001B240C0A52F
:108440004001824A001892420E24021892421024DF
:1084500004189242122406189242142408189242D8
:1084600016240A18924218240C1892421A240E1844
:10847000824B10181A17304121835F4280234F939B
:108480004C38F2F0FEFF3C095E4280234E4E5F42C4
:1084900081234F4F8F100FDE3F900203092C3F9036
:1084A00000032B280E430F43B012D28321533041D7
:1084B0003F9082060D283F90000951243F902109EA
:1084C0006E243F9080086424F2D220092153304169
:1084D0003F90800625285F4283236F93D5247F90A9
:1084E0000300BF28D8247F902200EE233E402200C4
:1084F0003F401C8BB012D283D93F3F90820017249B
:108500003F908300682C3F908000DE2B2E433F403D
:108510002024B012D28321533041D2D33C09B43F3E
:108520003F900005D123D24282233F09BB3F5E42E8
:1085300084234E4E5F4285234F4F8F100FDE3F90B6
:108540008100C2235E42C8233EF21F4301200F4335
:10855000814F00002E430F41B012D283A73FB012CB
:1085600024835E4282235F4283234F4F8F104EDF6E
:10857000C24E08240E430F43B012D2835F42082438
:108580004F934420B0122483F2F07F0063028E3FA9
:108590001E433F400824B012D283215330415E4233
:1085A00082234E4E5F4283234F4F8F100FDE3F904A
:1085B00002038A235E4286234E4E5F4287234F4F3B
:1085C0008F100FDE3F901400552CB2400A24062471
:1085D000824F0424793F3F900001762B3F900201A7
:1085E000612B3F90A10170235E4282234E4E5F4279
:1085F00083234F4F8F100FDE3F9003033E243E40F6
:1086000014003F400A24B012D283503F5F934E23A0
:10861000F2D080FF6302C243C8235F421E24C24FD0
:10862000C9234E4F7E52C24ECD237F501000C24F01
:108630001E24F2D01000C823F2404000CF23F240A5
:1086400080FFCA23F24080FFCE23F2D084FFC823EC
:10865000E2D32E09C243011CC243411CD2430B2466
:10866000253F5F9331233E4012003F405A8AB012AB
:10867000D2831C3F3F401400A83F3E4006003F40CD
:108680002224B012D283123F3E4022003F406C8A27
:10869000B012D2830B3F5E4282234E4E2E92142F95
:1086A0003F408E8A0E9305206E4FB012D283304029
:1086B000AC846D4F0F5D3E53FC230F93F523304088
:1086C000C8846F155F423E092FF222201F423209F3
:1086D0000E4F3E50EEFF3E900F0017280E4F3E50BB
:1086E000DCFF3E900D000F283F50CEFF3F900D0065
:1086F0000A2C5F015F534F4F5F0A3F5080236E4F3C
:108700007ED2CF4E0000691700135E02104E3C8AE5
:10871000F2D010003C09B0127884F2F0FBFF3E0961
:10872000D53FC24323098293042461205F4220097C
:108730007FD2C24F2009691700131B4204240B93F8
:108740004E245A4223093AF07F000B9A4E381942C0
:1087500006240D4A3E4070230F49B0125689095A2B
:10876000824906240B8A824B0424C2432309CB236B
:10877000B012F683C83FB0124A8369170013F2D0D3
:1087800010003C09F2F0BFFF3E091F4210093FF004
:10879000FFFE824F1009F24020003D0969170013C7
:1087A000B24011021209B2400003100982431409B9
:1087B0003F406A0A1F83FE231F4214090F93F623CA
:1087C0005F423E097FF09FFFC24F3E09F240C4FF67
:1087D0003D0969170013B0127884691700135F42CE
:1087E00022097FD2C24F22098E3F0A4BB03FB012FE
:1087F0009E83893F7F15F2E0400063021842200704
:108800001F42240719422A071A422E071B42220739
:108810001E4226071C422C071D423007C2930B2420
:1088200036240F580F590F5A5F070E5B0E5C0E5D12
:108830005E065D42C8233DF0200074203C40001CD1
:108840000D4C1D535B4C01008B110D5BCD4F010096
:108850004B4E7BF0F0FF8F104BDFCD4B02008E10A4
:10886000CD4E03005F4C01007F500300CC4F010050
:108870007F903C000C38F2404000CA235F42C8237E
:108880003FF0200052203F40001CCF4301001E4219
:1088900018241F421A241E5200241F620224824EF2
:1088A0000024824F0224829F162424381F9216240B
:1088B0001E34B01252821E4228071E5228241F4224
:1088C00032071F522A245D4223245D53C24D2324C4
:1088D0003DF00F000620824E2424824F26240F43B1
:1088E0000E43824E2824824F2A2478170013829E3A
:1088F0001424DF2F924210240024924212240224D6
:10890000B0125282C2930B24D627F2404000CA23F1
:108910005F42C8233FF020000B203F40001CCF43A4
:108920000100C93F3C40401C8B3F3F40401CAD3FD5
:108930003F40401CF43F0B120D930A247B4F7C4EAA
:108940004B9C04244F4B4E4C0F8E033C3D53F43F45
:108950000F433B4130414B150D936D240F9E6B240B
:10896000332C0C4E0CDF1CF31B240C4E0CEF1CF3B1
:1089700007202D9307280B4E1BF32C430C8B033C35
:108980000C4D013C1C430D8C0A4C094E0B4FFB490E
:1089900000001B533A53FB230B4F0B5C0E5C013C56
:1089A0000B4F0C4D5C030B24094C084E0A4BBA4884
:1089B00000002A533953FB235C020E5C0B5C1DF351
:1089C0003A24EB4E0000373C0E5D0C4F0C5D0B4C17
:1089D0000BDE1BF31B240B4C0BEE1BF306203D9010
:1089E000030003280B4E1BF3013C0B4D0D8B094E6E
:1089F0000A4C084B088C3A533953EA490000074A9D
:108A00000758F9233BE31B530C5B0E5B0A4D5A03DB
:108A10000D240B4A084E094C28832983A9480000DD
:108A20003B53FA230B8A5B020E5B0C5B1DF30324A2
:0C8A3000DC4EFFFFFFFF47173041001332
:108A3C002287DC863A87DC867687DC867E87DC8636
:108A4C00A087DC86DC86DC86DC86DC86D687120199
:108A5C00010100000008C016D927500001020301D3
:108A6C0009022200010100804609040000010300F4
:108A7C0000000921010100012222000705810340A9
:108A8C0000010403070424036800610066007400FD
:108A9C006D0061006E006E00230073006F006600B5
:108AAC007400770061007200650026034E006500BB
:108ABC0074007A007700650072006B0061006E0034
:108ACC0061006C0079007300610074006F0072002B
:108ADC003E03680065006E00720069006B002E009A
:108AEC0068006100660074006D0061006E006E002D
:108AFC00400067006D00610069006C002E0063008F
:108B0C006F006D003A00300030003500300000007E
:108B1C000600FF0901A1018501953F750809018136
:108B2C0002850295130902B102850395050903B16B
:0C8B3C0002C01012101211101210129A38
:10FF8000FFFFFFFFFFFFFFFFFFFFFFFFFFFFFFFF81
:10FF9000FFFFFFFFFFFFFFFFFFFFFFFFFFFFFFFF71
:10FFA000FFFFFFFFFFFFFFFFFFFFFFFFFFFFFFFF61
:10FFB000FFFFFFFFFFFFFFFFFFFFFFFFFFFFFFFF51
:10FFC0001C821C821C821C821C821C821C821C8241
:10FFD0001C821C821C821C821C821C821C821C8231
:10FFE0001C821C821C82C2861C821C82F4871C829A
:10FFF0001C821C821C821C821C821C821C8200802F
:040000030000800079
:00000001FF
